:020000040800F2
:100000000006022001020008850F0008050F000805
:100010005D0F0008050F0008310F000803020008FB
:10002000030200080302000803020008ED2800088C
:10003000030200080302000803020008030200088C
:10004000030200080302000803020008030200087C
:100050000302000803020008513A0008793A000838
:10006000A13A0008C93A0008F13A00080302000862
:10007000030200080302000803020008030200084C
:10008000030200080302000803020008030200083C
:10009000030200080302000803020008193B0008DD
:1000A000030200080302000803020008030200081C
:1000B000293C0008030200080302000803020008AC
:1000C00003020008030200080302000803020008FC
:1000D0000302000803020008ED3B0008013C000891
:1000E0007D3B000803020008030200080302000829
:1000F00003020008030200080302000803020008CC
:1001000003020008030200080302000803020008BB
:1001100003020008030200080302000803020008AB
:10012000030200080302000803020008030200089B
:10013000030200080302000803020008030200088B
:10014000030200080302000803020008A1300008AF
:10015000030200080302000803020008030200086B
:10016000030200080302000803020008030200085B
:10017000030200080302000803020008030200084B
:100180000302000803020008153C000803020008EF
:10019000030200080302000803020008030200082B
:1001A000030200080302000803020008030200081B
:1001B000030200080302000803020008030200080B
:1001C00003020008030200080302000803020008FB
:1001D00003020008030200080302000803020008EB
:1001E00003020008030200080302000803020008DB
:1001F00003020008030200080302000803020008CB
:1002000002E000F000F8FEE772B63A4880F3088892
:10021000394880F3098839484EF60851CEF200017A
:10022000086040F20000CCF200004EF63471CEF2CD
:1002300000010860BFF34F8FBFF36F8F40F20000E3
:10024000C0F2F0004EF68851CEF200010860BFF314
:100250004F8FBFF36F8F4FF00000E1EE100A4EF6A4
:100260003C71CEF200010860062080F31488BFF3D1
:100270006F8F02F0F9FB02F09BFB03F08BFA4FF05B
:1002800055301F491B4A91423CBF41F8040BFAE725
:100290001C49194A91423CBF41F8040BFAE71A493C
:1002A0001A4A1B4B9A423EBF51F8040B42F8040B0A
:1002B000F8E700201749184A91423CBF41F8040B67
:1002C000FAE702F0B3FB03F0C5FA144C144DAC424C
:1002D00003DA54F8041B8847F9E700F041F8114CA1
:1002E000114DAC4203DA54F8041B8847F9E702F0D9
:1002F0009BBB000000060220002202200000000834
:1003000000000220000602207040000800220220A7
:1003100068220220682202205039022000020008D0
:100320000002000800020008000200082DE9F04F5A
:100330002DED108AC1F80CD0D0F80CD0BDEC108A8D
:10034000BDE8F08F002383F311882846A0470020E2
:1003500001F0D6FEFEE701F051FE00DFFEE70000EF
:1003600038B502F0ABFA40B1174B6FF07F010022B5
:1003700059720E211A729972DA7202F075FA0546F4
:1003800002F0AAFA0446D0B9104B9D4219D00133AD
:100390009D4241F2883512BF044600250124002009
:1003A00002F06CFA0CB100F079F800F04DFD00F0AD
:1003B00007FC284600F0FCF800F070F8F9E700258B
:1003C000EDE70546EBE700BF00220220010007B081
:1003D00008B500F0C1FBA0F120035842584108BD08
:1003E00007B541F21203022101A8ADF8043000F074
:1003F000D1FB03B05DF804FB38B5202383F31188EB
:100400001748C3680BB101F001FF0023154A4FF4F0
:100410007A71134801F0BEFE002383F31188124C59
:10042000236813B12368013B2360636813B16368D9
:10043000013B63600D4D2B7833B963687BB90220B3
:1004400000F084FC322363602B78032B07D16368B0
:100450002BB9022000F07AFC4FF47A73636038BD48
:1004600068220220F9030008842302207C22022053
:10047000084B187003280CD8DFE800F008050208C4
:10048000022000F061BC022000F05CBC024B0022A4
:100490005A6070477C22022084230220F8B53F4B2B
:1004A0003F4A1C461968013177D004339342F9D191
:1004B0006268A24271D33B4B9B6803F1006303F572
:1004C000C0339A4269D2002000F094FB0220FFF76B
:1004D000CFFF354B00211A6C19641A6E19661A6E1B
:1004E0005A6C59645A6E59665A6E5A6942F08002C3
:1004F0005A615A6922F080025A615A691A6942F0B7
:1005000000521A611A6922F000521A611B6972B610
:100510004FF0E023C3F8084DD4E90004BFF34F8F38
:10052000BFF36F8F214AC2F88410BFF34F8F536916
:1005300023F480335361BFF34F8FD2F8803043F6FA
:10054000E076C3F3C905C3F34E335B0103EA060C3F
:1005500029464CEA81770139C2F87472F9D2203BFE
:1005600013F1200FF2D1BFF34F8FBFF36F8FBFF3A3
:100570004F8FBFF36F8F536923F400335361002310
:10058000C2F85032BFF34F8FBFF36F8F202383F336
:100590001188854680F308882047F8BD008001084F
:1005A00020800108002202200038024000ED00E017
:1005B0002DE9F04F93B0B44B2022FF2100900AA800
:1005C0009D6800F0EBFBB14A1378A3B90121B04854
:1005D0001170C360202383F31188C3680BB101F04D
:1005E00015FE0023AB4A4FF47A71A94801F0D2FD01
:1005F000002383F31188009B13B1A74B009A1A6064
:10060000A64A1378032B03D000231370A24A536029
:100610004FF0000A009CD3465646D146012000F018
:1006200093FB24B19C4B1B68002B00F0268200201A
:1006300000F092FA0390039B002BF2DB012000F004
:1006400081FB039B213B1F2BE8D801A252F823F02A
:10065000D1060008F90600088D0700081D060008ED
:100660001D0600081D0600081F080008EF09000805
:10067000090900086B09000893090008B909000876
:100680001D060008CB0900081D0600083D0A0008E9
:10069000710700081D060008810A0008DD06000831
:1006A000710700081D0600086B0900081D060008F8
:1006B0001D0600081D0600081D0600081D0600088E
:1006C0001D0600081D0600081D0600088D0700080D
:1006D0000220FFF77DFE002840F0F981009B0221F7
:1006E00005A8BAF1000F08BF1C4641F21233ADF85D
:1006F000143000F04FFA91E74FF47A7000F02CFAC2
:10070000071EEBDB0220FFF763FE0028E6D0013F67
:10071000052F00F2DE81DFE807F0030A0D10133623
:100720000523042105A8059300F034FA17E00421FD
:100730005548F9E704215A48F6E704215948F3E7F8
:100740004FF01C08404608F1040800F055FA042157
:10075000059005A800F01EFAB8F12C0FF2D1012087
:100760004FF0000900FA07F747EA0B0B5FFA8BFB23
:1007700000F060FB26B10BF00B030B2B08BF00242D
:10078000FFF72EFE4AE704214748CDE7002EA5D00B
:100790000BF00B030B2BA1D10220FFF719FE07462C
:1007A00000289BD00120002600F024FA0220FFF749
:1007B0005FFE5FFA86F8404600F02CFA0446B0B1BE
:1007C000039940460136A1F140025142514100F0E7
:1007D00031FA0028EDD1BA46044641F21213022143
:1007E00005A83E46ADF8143000F0D4F916E72546CA
:1007F0000120FFF73DFE244B9B68AB4207D92846FA
:1008000000F0FAF9013040F067810435F3E7002584
:10081000224BBA463E461D701F4B5D60A8E7002E76
:100820003FF45CAF0BF00B030B2B7FF457AF0220B0
:10083000FFF71EFE322000F08FF9B0F10008FFF63E
:100840004DAF18F003077FF449AF0F4A08EB0503DB
:10085000926893423FF642AFB8F5807F3FF73EAFD4
:10086000124BB845019323DD4FF47A7000F074F910
:100870000390039A002AFFF631AF039A0137019BD8
:1008800003F8012BEDE700BF0022022080230220A5
:1008900068220220F9030008842302207C2202201F
:1008A00004220220082202200C22022080220220A0
:1008B000C820FFF78DFD074600283FF40FAF1F2D1E
:1008C00011D8C5F120020AAB25F003008449424546
:1008D000184428BF4246019200F03AFA019AFF21DB
:1008E0007F4800F05BFA4FEAA803C8F387027C490F
:1008F0002846019300F05AFA064600283FF46DAFEF
:10090000019B05EB830533E70220FFF761FD00281B
:100910003FF4E4AE00F0BAF900283FF4DFAE002760
:10092000B846704B9B68BB4218D91F2F11D80A9B41
:1009300001330ED027F0030312AA134453F8203CCE
:1009400005934046042205A9043700F01DFB8046AC
:10095000E7E7384600F050F90590F2E7CDF814804B
:10096000042105A800F016F902E70023642104A879
:10097000049300F005F900287FF4B0AE0220FFF7E1
:1009800027FD00283FF4AAAE049800F067F905900F
:10099000E6E70023642104A8049300F0F1F800289E
:1009A0007FF49CAE0220FFF713FD00283FF496AEC3
:1009B000049800F063F9EAE70220FFF709FD002838
:1009C0003FF48CAE00F072F9E1E70220FFF700FD82
:1009D00000283FF483AE05A9142000F06DF9074606
:1009E0000421049004A800F0D5F83946B9E7322074
:1009F00000F0B2F8071EFFF671AEBB077FF46EAED3
:100A0000384A07EB0903926893423FF667AE02202B
:100A1000FFF7DEFC00283FF461AE27F003074F44E8
:100A2000B9453FF4A5AE484609F1040900F0E4F8E1
:100A30000421059005A800F0ADF8F1E74FF47A70B5
:100A4000FFF7C6FC00283FF449AE00F01FF900286C
:100A500044D00A9B01330BD008220AA9002000F0E1
:100A6000A5F900283AD02022FF210AA800F096F923
:100A7000FFF7B6FC1C4801F049FB13B0BDE8F08F4E
:100A8000002E3FF42BAE0BF00B030B2B7FF426AEA6
:100A90000023642105A8059300F072F8074600289A
:100AA0007FF41CAE0220FFF793FC804600283FF441
:100AB00015AEFFF795FC41F2883001F027FB059851
:100AC00000F000FA46463C4600F0B4F9A6E50646BA
:100AD0004EE64FF0000901E6BA467EE637467CE670
:100AE0008022022000220220A08601002DE9F84F7A
:100AF0004FF47A7306460D46002402FB03F7DFF835
:100B00005080DFF8509098F900305FFA84FA5A1C50
:100B100001D0A34210D159F824002A463146036877
:100B2000D3F820B03B46D847854205D1074B01207A
:100B300083F800A0BDE8F88F0134042CE3D14FF412
:100B4000FA7001F0E3FA0020F4E700BFD02302209E
:100B500010220220143D0008002307B5024601219F
:100B60000DF107008DF80730FFF7C0FF20B19DF8A9
:100B7000070003B05DF804FB4FF0FF30F9E7000019
:100B80000A46042108B5FFF7B1FF80F00100C0B2AA
:100B9000404208BD074B0A4630B41978064B53F85B
:100BA0002140014623682046DD69044BAC4630BC39
:100BB000604700BFD0230220143D0008A08601003A
:100BC00070B50A4E00240A4D01F040FD30802868BF
:100BD0003388834208D901F033FD2B680444013384
:100BE000B4F5C03F2B60F2D370BD00BFD22302200A
:100BF0008C23022001F0ECBD00F1006000F5C03054
:100C00000068704700F10060920000F5C03001F00C
:100C10006BBD0000054B1A68054B1B889B1A83426D
:100C200002D9104401F00CBD002070478C23022033
:100C3000D223022038B50446074D29B12868204444
:100C4000BDE8384001F01CBD2868204401F000FDDB
:100C50000028F3D038BD00BF8C23022010F003031E
:100C600009D1B0F5846F04D200F10050A0F57120D5
:100C70000368184670470023FBE7000000F10050AE
:100C8000A0F57120D0F8200470470000064991F8C3
:100C9000243033B100230822086A81F82430FFF79A
:100CA000B1BF0120704700BF90230220014B18689C
:100CB000704700BF002004E0204B0246F0B51868E2
:100CC0001F4BC0F30B06000C1F885D68BE4293F9F2
:100CD000084022D09F89BE4221D01F8BBE4206D140
:100CE00002240C2505FB04335D6893F90840B0F538
:100CF000805F16D041F20103984208BF5A24013A9E
:100D0000013D0B460A4493420DD215F9016F581C60
:100D10005EB1034600F8016CF5E70024E1E7012429
:100D2000DFE74124EBE7184605E02C2590421D70D3
:100D300001D2981C5C70401AF0BD00BF002004E096
:100D40001422022070470000704700007047000026
:100D5000002310B5934203D0CC5CC4540133F9E7AF
:100D600010BD0000013810B510F9013F3BB191F9F9
:100D700000409C4203D11AB10131013AF4E71AB1A3
:100D800091F90020981A10BD1046FCE70346024670
:100D9000D01A12F9011B0029FAD170470244034608
:100DA000934202D003F8011BFAE770472DE9F8439C
:100DB0001F4D14460746884695F8242052BBDFF89D
:100DC00070909CB395F824302BB92022FF2148461F
:100DD0002F62FFF7E3FF95F824004146C0F10802B7
:100DE00005EB8000A24228BF2246D6B29200FFF750
:100DF000AFFF95F82430A41B17441E449044E4B27E
:100E0000F6B2082E85F82460DBD1FFF73FFF0028FB
:100E1000D7D108E02B6A03EB82038342CFD0FFF7E0
:100E200035FF0028CBD10020BDE8F8830120FBE787
:100E300090230220024B1A78024B1A70704700BFB1
:100E4000D023022010220220F8B5184C184800F0D8
:100E50006BFC2146164800F093FC24681548E26EAE
:100E6000154ED2F80438154D43F00203104FC2F866
:100E7000043801F04BF92046114900F089FDE26E7B
:100E80000424D2F8043823F00203C2F804384FF4E3
:100E9000E133336055F8040BB84202D0314600F01C
:100EA000A3FB013C14F0FF04F4D1F8BD2C3E000874
:100EB000D02C022040420F00B8230220143D00082D
:100EC000343E000838B50B4B04461A780A4B53F8E9
:100ED00022500A4B9D420CD0094B00211822184683
:100EE000FFF75CFF046001462846BDE8384000F08B
:100EF0007BBB38BDD0230220143D0008D02C02203B
:100F0000B823022000B59BB0EFF309816822684640
:100F1000FFF71EFFEFF30583044B9A6BDA6A9A6AB8
:100F20009A6A9A6A9A6A9A6A9B6AFEE700ED00E0FA
:100F300000B59BB0EFF3098168226846FFF708FF10
:100F4000EFF30583044B9A6B9A6A9A6A9A6A9A6AD3
:100F50009A6A9B6AFEE700BF00ED00E000B59BB017
:100F6000EFF3098168226846FFF7F2FEEFF305838D
:100F7000034B5A6B9A6A9A6A9A6A9A6A9B6AFEE764
:100F800000ED00E0FEE7000030B50A44084D914254
:100F90000DD011F8013B5840082340F30004013BF9
:100FA0002C4013F0FF0384EA5000F6D1EFE730BD88
:100FB0002083B8ED026843681143016003B118470C
:100FC00070470000024A136843F0C0031360704783
:100FD00000440040024A136843F0C00313607047A6
:100FE00000480040024A136843F0C0031360704792
:100FF0000078004037B5274C274D204600F0E8FA2E
:1010000004F11400009400234FF48072234900F08F
:10101000A9F94FF48072224904F138000094214B61
:1010200000F022FA204BC4E91735204C204600F08E
:10103000CFFA04F11400009400234FF480721C498D
:1010400000F090F94FF480721A4904F138000094CE
:10105000194B00F009FA194BC4E91735184C204612
:1010600000F0B6FA04F1140000234FF48072154921
:10107000009400F077F9144B4FF48072134904F197
:101080003800009400F0F0F9114BC4E9173503B0B3
:1010900030BD00BFD423022080F937031825022079
:1010A00018280220C50F00080044004040240220F8
:1010B0001826022018290220D50F000800480040F9
:1010C000AC24022018270220E50F0008182A02206D
:1010D00000780040037C30B52E4C002918BF0C4628
:1010E000012B13D12C4B98420AD12C4B1A6C42F491
:1010F00000321A641A6E42F400321A661B6E05E062
:10110000274B98422FD0274B984235D02268036E48
:10111000C16D03EB52038466B3FBF2F362681504FE
:1011200042BF23F0070503F0070343EA4503CB6002
:10113000A36843F040034B60E36843F001038B6016
:1011400042F4967343F001030B604FF0FF330B62E0
:10115000510505D512F0102217D0B2F1805F16D0DC
:1011600080F8643030BD0D4B1A6C42F480221A6452
:101170001A6E42F48022C0E7084B1A6C42F080429B
:101180001A641A6E42F08042B7E77F23E8E73F23F4
:10119000E6E700BF243D0008D423022000380240C7
:1011A00040240220AC2402202DE9F047C66D0546FC
:1011B0003768F4692107346219D014F0080118BFA8
:1011C0008021E20748BF41F02001A3074FF0200330
:1011D00048BF41F04001600748BF41F4807183F38C
:1011E0001188281DFFF7E6FE002383F31188E2052E
:1011F0000AD5202383F311884FF40071281DFFF7CF
:10120000D9FE002383F311884FF020094FF0000A24
:1012100014F0200838D13B0616D54FF0200905F10F
:10122000380A200610D589F31188504600F050F98D
:10123000002836DA0821281DFFF7BCFE27F08003BE
:101240003360002383F31188790614D5620612D522
:10125000202383F31188D5E913239A4208D12B6CFC
:1012600033B127F040071021281DFFF7A3FE376098
:10127000002383F31188E30618D5AA6E1369ABB176
:101280005069BDE8F047184789F31188736A28460A
:1012900095F86410194000F0B5F98AF31188F469E3
:1012A000B6E7B06288F31188F469BAE7BDE8F08761
:1012B000F8B51546826804460B46AA4200D28568F6
:1012C000A1692669761AB5420BD218462A46FFF75D
:1012D0003FFDA3692B44A3612846A3685B1BA36061
:1012E000F8BD0CD9AF1B18463246FFF731FD3A4620
:1012F000E1683044FFF72CFDE3683B44EBE7184618
:101300002A46FFF725FDE368E5E70000836893427E
:10131000F7B50446154600D28568D4E90460361A4C
:10132000B5420BD22A46FFF713FD63692B44636174
:101330002846A3685B1BA36003B0F0BD0DD93246FD
:10134000AF1B0191FFF704FD01993A46E068314473
:10135000FFF7FEFCE3683B44E9E72A46FFF7F8FCA9
:10136000E368E4E710B50A440024C361029B84608B
:10137000C16002610362C0E90000C0E9051110BD4F
:1013800008B5D0E90532934201D1826882B98268FA
:10139000013282605A1C426119700021D0E9043286
:1013A0009A4224BFC368436100F0CCFE002008BD10
:1013B0004FF0FF30FBE7000070B5202304460E46D7
:1013C00083F31188A568A5B1A368A269013BA36056
:1013D000531CA36115782269934224BFE368A3617B
:1013E000E3690BB120469847002383F31188284610
:1013F00007E03146204600F095FE0028E2DA85F34A
:10140000118870BD2DE9F74F04460E4617469846E1
:10141000D0F81C904FF0200A8AF311884FF0000B8F
:10142000154665B12A4631462046FFF741FF03467F
:1014300060B94146204600F075FE0028F1D0002337
:1014400083F31188781B03B0BDE8F08FB9F1000F6A
:1014500003D001902046C847019B8BF31188ED1AF9
:101460001E448AF31188DCE7C160C361009B82607F
:101470000362C0E905111144C0E900000161704731
:10148000F8B504460D461646202383F31188A76855
:10149000A7B1A368013BA36063695A1C62611D7018
:1014A000D4E904329A4224BFE3686361E3690BB173
:1014B00020469847002080F3118807E031462046F7
:1014C00000F030FE0028E2DA87F31188F8BD000052
:1014D000D0E9052310B59A4201D182687AB98268B1
:1014E0000021013282605A1C82611C7803699A4291
:1014F00024BFC368836100F025FE204610BD4FF075
:10150000FF30FBE72DE9F74F04460E461746984695
:10151000D0F81C904FF0200A8AF311884FF0000B8E
:10152000154665B12A4631462046FFF7EFFE0346D1
:1015300060B94146204600F0F5FD0028F1D00023B7
:1015400083F31188781B03B0BDE8F08FB9F1000F69
:1015500003D001902046C847019B8BF31188ED1AF8
:101560001E448AF31188DCE7026843681143016076
:1015700003B11847704700001430FFF743BF000065
:101580004FF0FF331430FFF73DBF00003830FFF756
:10159000B9BF00004FF0FF333830FFF7B3BF000092
:1015A0001430FFF709BF00004FF0FF311430FFF790
:1015B00003BF00003830FFF763BF00004FF0FF3279
:1015C0003830FFF75DBF000000207047FFF712BD05
:1015D000044B036000234360C0E90233012303741A
:1015E000704700BF3C3D000810B52023044683F33C
:1015F0001188FFF76FFD02232374002383F3118802
:1016000010BD000038B5C36904460D461BB904215E
:101610000844FFF7A9FF294604F11400FFF7B0FEC4
:10162000002806DA201D4FF48061BDE83840FFF73E
:101630009BBF38BD026843681143016003B118477E
:101640007047000013B5446BD4F8A4381A681178B9
:10165000042915D1217C022912D11979012312897B
:101660008B4013420CD101A904F14C0001F098FF0A
:10167000D4F8A4480246019B2179206800F0D4F9EF
:1016800002B010BD143001F01BBF00004FF0FF335B
:10169000143001F015BF00004C3001F0EDBF000028
:1016A0004FF0FF334C3001F0E7BF0000143001F081
:1016B000E9BE00004FF0FF31143001F0E3BE00003E
:1016C0004C3001F0B9BF00004FF0FF324C3001F058
:1016D000B3BF000000207047D0F8A4381A6810B5D6
:1016E00011780446042917D1017C022914D15979B3
:1016F000012352898B4013420ED1143001F07CFE3D
:10170000024648B1D4F8A4484FF480736179206848
:10171000BDE8104000F076B910BD0000406BFFF747
:10172000DBBF0000704700007FB5124B0125042687
:10173000044603600023057400F1840243602946D7
:10174000C0E902330C4B0290143001934FF48073C4
:10175000009601F02DFE094B04F29442294604F153
:101760004C000294CDE900634FF4807301F0F4FE65
:1017700004B070BD643D00081D1700084516000840
:101780000B68202282F311880A7903EB820210622F
:101790004A790D3243F822008A7912B103EB8203B1
:1017A00018620223C0F8A4180374002383F311887D
:1017B0007047000038B5037F044613B190F85430E9
:1017C000ABB90125201D0221FFF734FF04F11400FD
:1017D0006FF00101257700F0C1FC04F14C0084F8A2
:1017E00054506FF00101BDE8384000F0B7BC38BD7F
:1017F00010B5012104460430FFF71CFF00232377B6
:1018000084F8543010BD000038B50446002514306B
:1018100001F0E6FD04F14C00257701F0B5FE201D36
:1018200084F854500121FFF705FF2046BDE83840F9
:10183000FFF752BF90F85C3003F06003202B06D115
:1018400090F85D200023212A03D81F2A06D8002003
:101850007047222AFBD1C0E9143303E0034A026532
:101860000722426583650120704700BF38220220AD
:10187000D0F8A43837B51A680446117804291AD16B
:10188000017C022917D11979012312898B40134257
:1018900011D100F14C05284601F036FF58B101A9DD
:1018A000284601F07DFED4F8A4480246019B217928
:1018B000206800F0B9F803B030BD000000EB8103F0
:1018C000F0B51E6A85B004460D46FEB1202383F3B1
:1018D000118804EB8507301D0821FFF7ABFEFB687C
:1018E00006F14C005B691B681BB1019001F066FEBC
:1018F000019803A901F054FE024648B1039B294612
:10190000204600F091F8002383F3118805B0F0BD64
:10191000FB685A691268002AF5D01B8A013B134004
:10192000F1D104F15C02EAE70D3138B550F82140FD
:10193000DCB1202383F31188D4F8A42813685279EA
:1019400003EB8203DB689B695D6845B10421601885
:10195000FFF770FE294604F1140001F057FD204600
:10196000FFF7BAFE002383F3118838BD70470000EB
:1019700001F0F0B801232822002110B5044600F838
:10198000243BFFF70BFA0023C4E9013310BD00002C
:1019900038B50446202383F3118800254160C0E94F
:1019A0000355C0E90555C0E9075501F0E3F80223E6
:1019B000237085F3118838BD70B500EB81030546AF
:1019C00050690E461446DA6018B110220021FFF764
:1019D000E5F9A06918B110220021FFF7DFF93146BF
:1019E0002846BDE8704001F08FB90000826802F01F
:1019F000011282600022C0E90422C0E906220262CC
:101A000001F00EBAF0B4012500EB810447898D4046
:101A1000E4683D43A469458123600023A2606360BC
:101A2000F0BC01F029BA0000F0B4012500EB8104FC
:101A300007898D40E4683D43646905812360002384
:101A4000A2606360F0BC01F0A3BA000070B502238D
:101A50000025044603704566056280F84C50C0E9D5
:101A60000255C0E90455C0E9065501F0E9F863687C
:101A70001B6823B129462046BDE87040184770BD59
:101A8000037880F868300523037043681B6810B53D
:101A900004460BB1042198470023A36010BD000049
:101AA00090F86820436802701B680BB10521184745
:101AB0007047000070B590F84C30044613B1002315
:101AC00080F84C3004F15C02204601F0CBF96368E9
:101AD0009B68B3B994F85C3013F0600535D00021F1
:101AE000204601F031FC0021204601F023FC636810
:101AF0001B6813B1062120469847062384F84C3012
:101B000070BD204698470028E4D0B4F86230626D7A
:101B10009A4288BF636594F95C30656D002B4FF085
:101B2000200380F20381002D00F0F280092284F866
:101B30004C2083F3118800212046D4E91423FFF7B9
:101B400073FF002383F31188DAE794F85D2003F034
:101B50007F0343EA022340F20232934200F0C58041
:101B600021D8B3F5807F48D00DD8012B3FD0022B70
:101B700000F09380002BB2D104F1640222650222AE
:101B80006265A365C1E7B3F5817F00F09B80B3F583
:101B9000407FA4D194F85E30012BA0D1B4F864301A
:101BA00043F0020332E0B3F5006F4DD017D8B3F520
:101BB000A06F31D0A3F5C063012B90D86368204695
:101BC00094F85E205E6894F85F10B4F86030B04717
:101BD000002884D043682365036863651AE0B3F581
:101BE000106F36D040F6024293427FF478AF5C4BE0
:101BF0002365022363650023C3E794F85E30012B5D
:101C00007FF46DAFB4F8643023F00203A4F86430BD
:101C1000C4E91455A56578E7B4F85C30B3F5A06F56
:101C20000ED194F85E30204684F8663001F060F8FA
:101C300063681B6813B10121204698470323237072
:101C40000023C4E914339CE704F1670323650123EF
:101C5000C3E72378042B10D1202383F31188204677
:101C6000FFF7C4FE85F311880321636884F8675089
:101C700021701B680BB12046984794F85E30002B0A
:101C8000DED084F867300423237063681B68002B60
:101C9000D6D0022120469847D2E794F860302046FB
:101CA0001D0603F00F010AD501F0CEF8012804D07B
:101CB00002287FF414AF2B4B9AE72B4B98E701F0E7
:101CC000B5F8F3E794F85E30002B7FF408AF94F892
:101CD000603013F00F01B3D01A06204602D501F090
:101CE00047FBADE701F03AFBAAE794F85E30002B22
:101CF0007FF4F5AE94F8603013F00F01A0D01B060E
:101D0000204602D501F020FB9AE701F013FB97E78C
:101D1000142284F84C2083F311882B462A46294646
:101D20002046FFF76FFE85F31188E9E65DB11522C5
:101D300084F84C2083F3118800212046D4E9142331
:101D4000FFF760FEFDE60B2284F84C2083F3118838
:101D50002B462A4629462046FFF766FEE3E700BFEA
:101D6000943D00088C3D0008903D000838B590F87F
:101D70004C300446002B3ED0063BDAB20F2A34D852
:101D80000F2B32D8DFE803F03731310822323131FE
:101D90003131313131313737456DB0F862309D42E4
:101DA00014D2C3681B8AB5FBF3F203FB12556DB95D
:101DB000202383F311882B462A462946FFF734FE59
:101DC00085F311880A2384F84C300EE0142384F83C
:101DD0004C30202383F31188002320461A461946ED
:101DE000FFF710FE002383F3118838BD836D03B124
:101DF00098470023E7E70021204601F0A5FA0021DB
:101E0000204601F097FA63681B6813B1062120464B
:101E100098470623D7E7000010B590F84C300446E9
:101E2000142B29D017D8062B05D001D81BB110BD13
:101E3000093B022BFBD80021204601F085FA002146
:101E4000204601F077FA63681B6813B1062120462B
:101E50009847062319E0152BE9D10B2380F84C3065
:101E6000202383F3118800231A461946FFF7DCFD6F
:101E7000002383F31188DAE7C3689B695B68002B52
:101E8000D5D1836D03B19847002384F84C30CEE759
:101E9000024B0022C3E900339A607047182B0220DE
:101EA000002382680374054B1B6899689142FBD23A
:101EB0005A6803604260106058607047182B022017
:101EC00008B5202383F31188037C032B05D0042B52
:101ED0000DD02BB983F3118808BD436900221A6025
:101EE0004FF0FF334361FFF7DBFF0023F2E7D0E958
:101EF000003213605A60F3E7002382680374054BD5
:101F00001B6899689142FBD85A6803604260106070
:101F100058607047182B0220054B1969087418681F
:101F2000026853601A60186101230374FEF7FEB95A
:101F3000182B02204B1C30B5044687B00A4D10D038
:101F40002B6901A8094A00F025F92046FFF7E4FFB4
:101F5000049B13B101A800F059F92B69586907B027
:101F600030BDFFF7D9FFF8E7182B0220C11E00088B
:101F700038B50C4D044641612B6981689A689142DD
:101F800003D8BDE83840FFF78BBF1846FFF7B4FF12
:101F900001232C61014623742046BDE83840FEF73A
:101FA000C5B900BF182B0220044B1A681B69906842
:101FB0009B68984294BF002001207047182B022094
:101FC00010B5084C236820691A6854602260012209
:101FD00023611A74FFF790FF01462069BDE81040A5
:101FE000FEF7A4B9182B022008B5FFF7DDFF18B1E2
:101FF000BDE80840FFF7E4BF08BD0000FFF7E0BF01
:10200000FEE7000010B50C4CFFF742FF00F0B4F8FB
:1020100080220A49204600F03BF8012344F8180CBE
:10202000037400F073FC002383F3118862B6044844
:10203000BDE8104000F04CB8402B0220983D00084D
:10204000A83D000800F01CB9EFF3118020B9EFF3B0
:102050000583202282F311887047000010B530B943
:10206000EFF30584C4F3080414B180F3118810BDA4
:10207000FFF7BAFF84F31188F9E70000034A5168BB
:1020800053685B1A9842FBD8704700BF001000E00D
:1020900082600222028270478368A3F17C0243F8C7
:1020A0000C2C026943F83C2C426943F8382C074A4F
:1020B00043F81C2CC268A3F1180043F8102C02222C
:1020C00003F8082C002203F8072C7047450300088A
:1020D00010B5202383F31188FFF7DEFF00210446AB
:1020E000FFF746FF002383F31188204610BD000050
:1020F000024B1B6958610F20FFF70EBF182B0220FF
:10210000202383F31188FFF7F3BF000008B50146D1
:10211000202383F311880820FFF70CFF002383F3AB
:10212000118808BD49B1064B42681B6918605A60A6
:10213000136043600420FFF7FDBE4FF0FF3070478F
:10214000182B02200368984206D01A68026050607B
:1021500018465961FFF7A4BE7047000038B5044621
:102160000D462068844200D138BD036823605C605E
:102170004561FFF795FEF4E7054B4FF0FF3103F1A2
:102180001402C3E905220022C3E90712704700BF09
:10219000182B022070B51C4E05460C46C0E90323DF
:1021A00001F0E4FA334653F8142F9A420DD130620D
:1021B0000A2C2CBF00190A302A60C5E90124C6E99F
:1021C0000555BDE8704001F0BFBA316A431AE31803
:1021D00038BF1C469368A34202D9081901F0C2FA1D
:1021E00073699A6894420CD85A68AC602B606A6034
:1021F00015609A685D60121B9A604FF0FF33F361BF
:1022000070BDA41A1B68ECE7182B022038B51B4CD4
:10221000636998420DD08168D0E9003213605A603A
:102220000022C2609A680A449A604FF0FF33E3616B
:1022300038BD03682246002142F8143F93425A6099
:10224000C16003D1BDE8384001F086BA9A68816860
:10225000256A0A449A6001F089FA6369411B9A6809
:102260008A42E5D9AB181D1A206A092D98BF01F1E1
:102270000A02BDE83840104401F074BA182B02205D
:102280002DE9F041184C002704F11406656901F0AE
:102290006DFA236AAA68C11A8A4215D81344D5F880
:1022A0000C802362D5E9003213605A606369EF60E5
:1022B000B34201D101F050FA87F311882869C04771
:1022C000202383F31188E1E76169B14209D0134407
:1022D0001B1ABDE8F0410A2B2CBFC0180A3001F0D0
:1022E00041BABDE8F08100BF182B022000207047E2
:1022F000FEE70000704700004FF0FF30704700001D
:1023000002290CD0032904D00129074818BF002056
:102310007047032A05D8054800EBC20070470448FF
:1023200070470020704700BF903E000848220220FE
:10233000443E000870B59AB005460846144601A907
:1023400000F0C2F801A8FEF721FD431C0022C6B22E
:102350005B001046C5E9003423700323023404F8FF
:10236000013C01ABD1B202348E4201D81AB070BD2B
:1023700013F8011B013204F8010C04F8021CF1E708
:1023800008B5202383F311880348FFF771FA00236F
:1023900083F3118808BD00BFD02C022090F85C3078
:1023A00003F01F02012A07D190F85D200B2A03D108
:1023B0000023C0E9143315E003F06003202B08D19B
:1023C000B0F860302BB990F85D20212A03D81F2A7D
:1023D00004D8FFF72FBA222AEBD0FAE7034A0265A6
:1023E0000722426583650120704700BF3F2202201B
:1023F00007B5052917D8DFE801F0191603191920C8
:10240000202383F31188104A01210190FFF7D4FAA9
:10241000019802210D4AFFF7CFFA0D48FFF7F4F9B2
:10242000002383F3118803B05DF804FB202383F3BA
:1024300011880748FFF7BEF9F2E7202383F31188DC
:102440000348FFF7D5F9EBE7E43D0008083E000834
:10245000D02C022038B50C4D0C4C2A460C4904F106
:102460000800FFF767FF05F1CA0204F110000949EF
:10247000FFF760FF05F5CA7204F118000649BDE8D0
:102480003840FFF757BF00BFA8350220482202207E
:10249000C03D0008CD3D0008D83D000870B5044699
:1024A00008460D46FEF772FCC6B22046013403789A
:1024B0000BB9184670BD32462946FEF753FC00287A
:1024C000F3D10120F6E700002DE9F04705460C4660
:1024D000FEF75CFC2B49C6B22846FFF7DFFF08B1C8
:1024E0000A36F6B228492846FFF7D8FF08B1103659
:1024F000F6B2632E0BD8DFF88C80DFF88C90234F78
:10250000DFF894A02E7846B92670BDE8F0872946FA
:102510002046BDE8F04701F0DFBB252E2ED1072273
:1025200041462846FEF71EFC70B9194B224603F1BE
:10253000100153F8040B8B4242F8040BF9D11B78BD
:10254000073511341370DDE7082249462846FEF7A7
:1025500009FC98B9A21C0F4B197802320909C95D10
:1025600002F8041C13F8011B01F00F015345C95D6B
:1025700002F8031CF0D118340835C3E7013504F81C
:10258000016BBFE7B03E0008D83D0008CA3E000816
:10259000B83E000820F4F01F2CF4F01FBFF34F8F5B
:1025A000024AD368DB03FCD4704700BF003C024002
:1025B00008B5074B1B7853B9FFF7F0FF054B1A69B5
:1025C000002A04DA044A5A6002F188325A6008BDCF
:1025D00006380220003C02402301674508B5054B40
:1025E0001B7833B9FFF7DAFF034A136943F000435E
:1025F000136108BD06380220003C02400B28F0B5EC
:1026000016D80C4C0C4923787BB90E460B4D0C2385
:102610004FF00062013B55F8047B46F8042B13F0A1
:10262000FF033A44F6D10123237051F82000F0BD96
:102630000020FCE73838022008380220DC3E000881
:10264000014B53F820007047DC3E00080C20704717
:102650000B2810B5044601D9002010BDFFF7CEFFAE
:10266000064B53F824301844C21A0BB90120F4E782
:1026700012680132F0D1043BF6E700BFDC3E0008EF
:102680000B2838B5044628D8FFF7DEFC0546FFF7CF
:1026900085FF2046FFF78CFF114AF323D360E30048
:1026A000DBB243F4007343F002031361136943F494
:1026B00080331361FFF772FFFFF7A0FF094B53F858
:1026C000241000F0E9F82846FFF788FFFFF7C6FC62
:1026D0002046BDE83840FFF7BBBF002038BD00BF33
:1026E000003C0240DC3E000812F001032DE9F041FD
:1026F00005460E4614464BD18218B2F1026F61D8DE
:10270000314B1B6813F001035CD0FFF79DFC2F4F8A
:10271000FFF74EFFF323314640F20128FB60FFF73D
:102720003DFF032C18D824F001046D1A274E40F207
:1027300001180C44A14205EB010733692AD123F0AB
:1027400001033361FFF74AFFFFF788FC0120BDE872
:10275000F081043C0435E4E7AB07E4D13B6923F4A2
:1027600040733B613B6943EA08033B6151F8046BEA
:102770002E60BFF34F8FFFF711FF2B689E42E8D00A
:102780003B6923F001033B61FFF728FFFFF766FC7D
:102790000020DCE723F440733361336943EA080324
:1027A00033610B883B80BFF34F8FFFF7F7FE3F8805
:1027B000BFB231F8023BBB42BCD0336923F0010306
:1027C0003361E1E71846C2E700380240003C0240AE
:1027D000084908B50B7828B11BB9FFF7E9FE0123BA
:1027E0000B7008BD002BFCD00870BDE80840FFF757
:1027F000F5BE00BF063802200244074BD2B210B526
:10280000904200D110BD441C00B253F8200041F8A2
:10281000040BE0B2F4E700BF502800400F4B30B586
:102820001C6F240407D41C6F44F400741C671C6FD5
:1028300044F400441C670A4C02442368D2B243F4B7
:1028400080732360074B904200D130BD441C51F887
:10285000045B00B243F82050E0B2F4E700380240D5
:10286000007000405028004007B5012201A9002057
:10287000FFF7C2FF019803B05DF804FB13B50446EF
:10288000FFF7F2FFA04205D0012201A90020019428
:10289000FFF7C4FF02B010BD0144BFF34F8F064BDA
:1028A000884204D3BFF34F8FBFF36F8F7047C3F8D5
:1028B0005C022030F4E700BF00ED00E0002070472C
:1028C000034B1A681AB9034AD2F874281A60704781
:1028D0003C3802200030024008B5FFF7F1FF024B00
:1028E0001868C0F3407008BD3C380220EFF309833C
:1028F000054968334A6B22F001024A6383F3098871
:10290000002383F31188704700EF00E0202080F35C
:10291000118862B60D4B0E4AD96821F4E0610904B2
:10292000090C0A430B49DA60D3F8FC2042F08072AC
:10293000C3F8FC20084AC2F8B01F116841F0010139
:1029400011601022DA7783F82200704700ED00E072
:102950000003FA0555CEACC5001000E0202310B5E9
:1029600083F311880E4B5B6813F4006314D0F1EE0F
:10297000103AEFF309844FF08073683CE361094B30
:10298000DB6B236684F30988FFF70EFB10B1064B5F
:10299000A36110BD054BFBE783F31188F9E700BF86
:1029A00000ED00E000EF00E0570300085A030008C4
:1029B00070B5BFF34F8FBFF36F8F1A4A0021C2F873
:1029C0005012BFF34F8FBFF36F8F536943F400333F
:1029D0005361BFF34F8FBFF36F8FC2F88410BFF303
:1029E0004F8FD2F8803043F6E074C3F3C900C3F3CD
:1029F0004E335B0103EA0406014646EA817501395C
:102A0000C2F86052F9D2203B13F1200FF2D1BFF38C
:102A10004F8F536943F480335361BFF34F8FBFF33C
:102A20006F8F70BD00ED00E0FEE700000A4B0B4821
:102A30000B4A90420BD30B4BC11EDA1C121A22F028
:102A400003028B4238BF00220021FEF7A7B953F8DA
:102A5000041B40F8041BECE7D84000085039022062
:102A600050390220503902207047000070B5D0E97B
:102A70001B4300224FF0FF359E6804EB42135101C7
:102A8000D3F80009002805DAD3F8000940F08040A7
:102A9000C3F80009D3F8000B002805DAD3F8000BBF
:102AA00040F08040C3F8000B013263189642C3F82F
:102AB0000859C3F8085BE0D24FF00113C4F81C3882
:102AC00070BD00001D4B03EB8002D2F80CC02DE955
:102AD000F043DCF81420461CDD6ED2F800E005EB74
:102AE000063605EB4018516871450AD30122D5F826
:102AF000343802FA00F023EA0000C5F83408BDE8D3
:102B0000F083AEEB0103BCF81040A34228BF23467C
:102B1000D8F81849A4B2B3EB840FF0D89468A4F1A4
:102B2000040959F8047F3760A4EB09071F44042FF8
:102B3000F7D81C440B4494605360D4E7403802201B
:102B4000890141F02001016103699B06FCD4122038
:102B5000FFF794BA10B5054C2046FEF70BFF4FF077
:102B6000A043E366024B236710BD00BF403802203C
:102B7000303F000870B503780546012B50D12A4B31
:102B8000C46E98421BD1294B0E2143205A6B42F050
:102B900080025A635A6D42F080025A655A6D5A6932
:102BA00042F080025A615A6922F080025A615B69E0
:102BB00000F0E8FB1E4BE3601E4BC4F80038002316
:102BC000EE6EC4F8003EC02323604FF40413A363E9
:102BD0003369002BFCDA01230C203361FFF74EFA36
:102BE0003369DB07FCD41220FFF748FA3369002B66
:102BF000FCDA00262846A660FFF738FF6B68C4F8A9
:102C00001068DB68C4F81468C4F81C684BB90A4B38
:102C1000A3614FF0FF336361A36843F00103A36036
:102C200070BD064BF4E700BF403802200038024078
:102C30004014004003002002003C30C0083C30C07B
:102C4000F8B5C46E054600214FF000662046FFF738
:102C500077FF296F00234FF001128F684FF0FF308C
:102C6000C4F83438C4F81C2804EB431201339F42E3
:102C7000C2F80069C2F8006BC2F80809C2F8080B74
:102C8000F2D20B68EA6E6B676362102313611669F8
:102C900016F01006FBD11220FFF7F0F9D4F8003837
:102CA00023F4FE63C4F80038A36943F4402343F0DF
:102CB0001003A3610923C4F81038C4F814380A4B70
:102CC000EB604FF0C043C4F8103B084BC4F8003B26
:102CD000C4F81069C4F800396B6F03F1100243F4B3
:102CE00080136A67A362F8BD0C3F000840800010A3
:102CF000C26E90F86610D2F8003823F4FE6343EAFF
:102D00000113C2F8003870472DE9F84300EB810346
:102D1000C56E0C468046DA680FFA81F948011668DC
:102D200006F00306731E022B05EB41134FF0000162
:102D300094BFB604384EC3F8101B4FF0010104F1E4
:102D4000100398BF06F1805601FA03F3916998BF0A
:102D500006F5004600293AD0578A04F15801374356
:102D600049016F50D5F81C180B430021C5F81C38D9
:102D70002B180127C3F81019A7405369611E9BB394
:102D8000138A928B9B08012A88BF5343D8F874207A
:102D9000981842EA034301F140022146C8F8740042
:102DA000284605EB82025360FFF7CAFE08EB890054
:102DB000C3681B8A43EA845348341E4364012E517E
:102DC000D5F81C381F43C5F81C78BDE8F88305EB1F
:102DD0004917D7F8001B21F40041C7F8001BD5F8AC
:102DE0001C1821EA0303C0E704F13F030B4A2846FD
:102DF000214605EB83035A60FFF7A2FE05EB49105D
:102E0000D0F8003923F40043C0F80039D5F81C3855
:102E100023EA0707D7E700BF008000100004000284
:102E2000026F12684267FFF721BE00005831C36E7F
:102E300049015B5813F4004004D013F4001F0CBF89
:102E400002200120704700004831C36E49015B58E1
:102E500013F4004004D013F4001F0CBF0220012023
:102E60007047000000EB8101CB68196A0B681360A2
:102E70004B6853607047000000EB810330B5DD689C
:102E8000AA691368D36019B9402B84BF402313602B
:102E90006B8A1468C26E1C4402EB4110013C09B2FB
:102EA000B4FBF3F46343033323F0030343EAC44363
:102EB00043F0C043C0F8103B2B6803F00303012B21
:102EC0000ED1D2F8083802EB411013F4807FD0F80D
:102ED000003B14BF43F0805343F00053C0F8003B65
:102EE00002EB4112D2F8003B43F00443C2F8003B2E
:102EF00030BD00002DE9F041244D0446EE6E06EB96
:102F00004013D3F8087B3807C3F8087B0AD5D6F8F6
:102F10001438190706D505EB840321462846DB68DB
:102F20005B689847FA071FD5D6F81438DB071BD51E
:102F300005EB8403D968CCB98B69488A5A68B2FB1F
:102F4000F0F600FB16228AB91868DA6890420DD2B2
:102F5000121AC3E90024202383F311880B48214669
:102F6000FFF78AFF84F31188BDE8F081012303FA9B
:102F700004F26B8923EA02036B81CB68002BF3D048
:102F800021460248BDE8F041184700BF4038022002
:102F900000EB81034A0170B5DD68C36E6C69266879
:102FA000E66056BB1A444FF40020C2F810092A68A4
:102FB00002F00302012A0AB20ED1D3F8080803EB8B
:102FC000421410F4807FD4F8000914BF40F0805000
:102FD00040F00050C4F8000903EB4212D2F8000997
:102FE00040F00440C2F800090122D3F8340802FA84
:102FF00001F10143C3F8341870BD19B9402E84BFE4
:103000004020206020681A442E8A8419013CB4FBB9
:10301000F6F440EAC44040F00050C6E7F8B5044674
:103020001E48C56E05EB4413D3F80869F107C3F8D1
:10303000086917D5D5F81038DA0713D500EB8403E3
:10304000D9684B691F68DA68974218D2D21B0027EB
:103050001A605F60202383F311882146FFF798FFF1
:1030600087F31188330617D50123D5F83428A340F8
:10307000134211D02046BDE8F840FFF723BD0123DD
:1030800003FA04F2038923EA020303818B68002B0D
:10309000E8D021469847E5E7F8BD00BF4038022058
:1030A0002DE9F74FA24CE66E7569B3691D4015F422
:1030B0008058756107D02046FEF7C8FC03B0BDE814
:1030C000F04FFFF74BBC002D12DAD6F8003E9F07F9
:1030D00005D0D6F8003E23F00303C6F8003ED6F82C
:1030E0000438934823F00103C6F80438FEF7D8FCEF
:1030F000280505D58E48FFF7B9FC8D48FEF7C0FCC2
:10310000A9040CD5D6F8083813F0060FF36823F499
:1031100070530CBF43F4105343F4A053F3602A07D9
:1031200004D56368DB680BB181489847EB0200F176
:103130008A80AF0227D5D4F86C9000274FF0010A9F
:10314000DFF8ECB109EB4712D2F8003B03F440235F
:10315000B3F5802F11D1D2F8003B002B0DDA628934
:103160000AFA07F322EA0303638104EB8703DB68AF
:10317000DB6813B13946584698470137236FFFB2D1
:103180009B689F42DED9E80618D5E76E3A6AC2F31B
:103190000A1002F00F0302F4F012B2F5802F00F0D3
:1031A0009C80B2F5402F09D104EB8303002207F580
:1031B0008057DB681B6A904240F082802B03D6F870
:1031C00018481DD5E70302D50020FFF793FEA6039C
:1031D00002D50120FFF78EFE600302D50220FFF723
:1031E00089FE210302D50320FFF784FEE20202D507
:1031F0000420FFF77FFEA30202D50520FFF77AFE29
:103200006F037FF55BAFE60702D50020FFF706FFEF
:10321000A50702D50120FFF701FF600702D50220B4
:10322000FFF7FCFE210702D50320FFF7F7FEE206B9
:1032300002D50420FFF7F2FEA3067FF53FAF05207D
:10324000FFF7ECFE3AE7E36E00274FF0010ADFF8E4
:10325000E0B00193236F5FFA87F99B6899453FF6C9
:1032600068AF019B03EB4913D3F8002902F4402215
:10327000B2F5802F22D1D3F80029002A1EDAD3F824
:10328000002942F09042C3F80029D3F80029002A0F
:10329000FBDB4946E06EFFF753FC22890AFA09F38B
:1032A00022EA0303238104EB8903DB689B6813B1E3
:1032B0004946584698474846FFF704FC0137C9E796
:1032C000910701D1D7F80080072A02F101029CBFC3
:1032D00003F8018B4FEA18286DE7023307F5805792
:1032E00004EB83025268D2F818C0DCF80820DCE94D
:1032F000001CA1EB0C0C002188420AD104EB8304D2
:1033000063689B699A6802449A605A6802445A60EA
:1033100054E711F0030F01D1D7F800808C4501F17B
:10332000010184BF02F8018B4FEA1828E4E700BFCF
:1033300040380220C36E03EB4111D1F8003B43F447
:103340000013C1F8003B7047C36E03EB4111D1F885
:10335000003943F40013C1F800397047C36E03EB22
:103360004111D1F8003B23F40013C1F8003B704732
:10337000C36E03EB4111D1F8003923F40013C1F8F7
:1033800000397047090100F16043012203F56143F0
:10339000C9B283F8001300F01F039A4043099B0051
:1033A00003F1604303F56143C3F880211A6070475D
:1033B00030B50433039C0172002104FB0325C16076
:1033C000C0E90653049B0363059BC0E90000C0E904
:1033D0000422C0E90842C0E90A11436330BD00007D
:1033E0000022416AC260C0E90411C0E90A226FF0FC
:1033F0000101FEF7B3BE0000D0E90432934201D1CF
:10340000C2680AB9181D7047002070470369196027
:103410000021C2680132C260C269134482699342CA
:10342000036124BF436A0361FEF78CBE38B50446CE
:103430000D46E3683BB162690020131D1268A36268
:103440001344E36207E0237A33B929462046FEF7A6
:1034500069FE0028EDDA38BD6FF00100FBE70000DF
:10346000C368C269013BC3604369134482699342E4
:10347000436124BF436A436100238362036B03B14A
:103480001847704770B52023044683F31188866A75
:103490003EB9FFF7CBFF054618B186F311882846E1
:1034A00070BDA36AE26A13F8015B9342A36202D380
:1034B0002046FFF7D5FF002383F31188EFE70000D4
:1034C0002DE9F84F04460E46174698464FF020095E
:1034D00089F311880025AA46D4F828B0BBF1000F63
:1034E00009D141462046FFF7A1FF20B18BF3118897
:1034F0002846BDE8F88FD4E90A12A7EB050B521A4B
:10350000934528BF9346BBF1400F1BD9334601F1C9
:10351000400251F8040B914243F8040BF9D1A36A1D
:10352000403640354033A362D4E90A239A4202D39D
:103530002046FFF795FF8AF31188BD42D8D289F360
:103540001188C9E730465A46FDF702FCA36A5E447B
:103550005D445B44A362E7E710B5029C043301724B
:1035600004FB0321C460C0E906130023C0E90A3349
:10357000039B0363049BC0E90000C0E90422C0E987
:103580000842436310BD0000026A6FF00101C2608F
:10359000426AC0E904220022C0E90A22FEF7DEBD29
:1035A000D0E904239A4201D1C26822B9184650F8E2
:1035B000043B0B607047002070470000C368002187
:1035C000C2690133C3604369134482699342436112
:1035D00024BF436A4361FEF7B5BD000038B5044619
:1035E0000D46E3683BB1236900201A1DA262E2691F
:1035F0001344E36207E0237A33B929462046FEF7F5
:1036000091FD0028EDDA38BD6FF00100FBE7000006
:1036100003691960C268013AC260C26913448269D1
:103620009342036124BF436A036100238362036BF7
:1036300003B118477047000070B520230D460446BB
:10364000114683F31188866A2EB9FFF7C7FF10B1C0
:1036500086F3118870BDA36A1D70A36AE26A013304
:103660009342A36204D3E16920460439FFF7D0FFF7
:10367000002080F31188EDE72DE9F84F04460D4650
:10368000904699464FF0200A8AF311880026B346E7
:10369000A76A4FB949462046FFF7A0FF20B187F33C
:1036A00011883046BDE8F88FD4E90A073A1AA8EB2A
:1036B0000607974228BF1746402F1BD905F1400344
:1036C00055F8042B9D4240F8042BF9D1A36A4036EB
:1036D0004033A362D4E90A239A4204D3E169204625
:1036E0000439FFF795FF8BF311884645D9D28AF349
:1036F0001188CDE729463A46FDF72AFBA36A3D44E7
:103700003E443B44A362E5E7D0E904239A4217D143
:10371000C3689BB1836A8BB1043B9B1A0ED01360C4
:10372000C368013BC360C3691A4483699A4202615A
:1037300024BF436A03610023836201231846704754
:103740000023FBE700F094B84FF080430022586359
:103750001A610222DA6070474FF080430022DA607B
:10376000704700004FF08043586370474FF080432C
:10377000586A70474B6843608B688360CB68C3604E
:103780000B6943614B6903628B6943620B68036099
:103790007047000008B52C4B40F2FF712B481A69A6
:1037A0000A431A611A6922F4FF6222F007021A61C1
:1037B0001A691A6B0A431A631A6D0A431A65244A76
:1037C0001B6D1146FFF7D6FF00F5806002F11C016A
:1037D000FFF7D0FF00F5806002F13801FFF7CAFF64
:1037E00000F5806002F15401FFF7C4FF00F580602E
:1037F00002F17001FFF7BEFF00F5806002F18C015D
:10380000FFF7B8FF00F5806002F1A801FFF7B2FFF3
:1038100000F5806002F1C401FFF7ACFF00F58060A5
:1038200002F1E001FFF7A6FF00F5806002F1FC0164
:10383000FFF7A0FF02F58C7100F58060FFF79AFF9B
:10384000BDE8084000F08AB800380240000002409D
:103850003C3F000808B500F01FFAFEF7D3FBFFF766
:103860002FF8BDE80840FEF7F5BD000070470000E6
:103870000F4B1A6C42F001021A641A6E42F00102F8
:103880001A660C4A1B6E936843F0010393604FF075
:1038900080436B229A624FF0FF32DA6200229A6113
:1038A0005A63DA605A6001225A611A60704700BF99
:1038B00000380240002004E04FF0804208B5116952
:1038C000D3680B40D9B29B076FEA0101116107D59C
:1038D000202383F31188FEF7B5FB002383F31188BF
:1038E00008BD00001B4B4FF0FF3000211A696FEA42
:1038F00042526FEA52521A611A69C2F30A021A61FD
:103900001A695A6958615A6959615A691A6A62F0A2
:1039100080521A621A6A02F080521A621A6A5A6A4D
:1039200058625A6A59625A6A0B4A106840F48070A9
:103930001060186F00F44070B0F5007F03D04FF4B2
:10394000803018671967536823F40073536000F0E0
:1039500073B900BF0038024000700040364B4FF48E
:103960004041364A1A64364A11601A6842F0010230
:103970001A601A689207FCD59A6822F003029A60CE
:103980002D4B9A6812F00C02FBD1196801F0F90175
:1039900019609A601A6842F480321A601A689003BB
:1039A000FCD55A6F42F001025A67234B5A6F9107B8
:1039B000FCD5244A5A601A6842F080721A60204B83
:1039C0005A685204FCD51A6842F480321A605A6868
:1039D000D003FCD51A6842F400321A60184A5368C2
:1039E0009903FCD5144B1A689201FCD5164A9A60CB
:1039F00040F20112C3F88C200022C3F8902040F25C
:103A00000733124A1360136803F00F03072BFAD130
:103A1000094B9A6842F002029A609A6802F00C021E
:103A2000082AFAD15A6C42F480425A645A6E42F41F
:103A300080425A665B6E70470038024000040010F6
:103A400000700040186C400900948838003C024027
:103A5000074A08B5536903F00103536123B1054ACE
:103A600013680BB150689847BDE80840FEF776BF71
:103A7000003C0140D0380220074A08B5536903F0E2
:103A80000203536123B1054A93680BB1D06898478C
:103A9000BDE80840FEF762BF003C0140D03802207C
:103AA000074A08B5536903F00403536123B1054A7B
:103AB00013690BB150699847BDE80840FEF74EBF47
:103AC000003C0140D0380220074A08B5536903F092
:103AD0000803536123B1054A93690BB1D069984734
:103AE000BDE80840FEF73ABF003C0140D038022054
:103AF000074A08B5536903F01003536123B1054A1F
:103B0000136A0BB1506A9847BDE80840FEF726BF1C
:103B1000003C0140D0380220164B10B55C6904F41B
:103B200078725A61A30604D5134A936A0BB1D06A1E
:103B30009847600604D5104A136B0BB1506B984739
:103B4000210604D50C4A936B0BB1D06B9847E20564
:103B500004D5094A136C0BB1506C9847A30504D5E2
:103B6000054A936C0BB1D06C9847BDE81040FEF746
:103B7000F5BE00BF003C0140D0380220194B10B503
:103B80005C6904F47C425A61620504D5164A136DDF
:103B90000BB1506D9847230504D5134A936D0BB1B3
:103BA000D06D9847E00404D50F4A136E0BB1506EE8
:103BB0009847A10404D50C4A936E0BB1D06E984778
:103BC000620404D5084A136F0BB1506F9847230461
:103BD00004D5054A936F0BB1D06F9847BDE81040EC
:103BE000FEF7BCBE003C0140D038022008B50348B7
:103BF000FDF7DAFABDE80840FEF7B0BED423022094
:103C000008B50348FDF7D0FABDE80840FEF7A6BEA8
:103C10004024022008B50348FDF7C6FABDE8084075
:103C2000FEF79CBEAC24022008B5FFF745FEBDE8B8
:103C30000840FEF793BE0000062108B50846FFF7CE
:103C4000A1FB06210720FFF79DFB06210820FFF7B7
:103C500099FB06210920FFF795FB06210A20FFF7B3
:103C600091FB06211720FFF78DFB06212820FFF787
:103C700089FB07211C20FFF785FB0C212620FFF77D
:103C800081FB0C212720FFF77DFB0C215220BDE892
:103C90000840FFF777BB000008B5FFF723FE00F0F0
:103CA0000DF8FDF793FCFDF763FEFDF73BFDFFF715
:103CB000DDFDBDE80840FFF745BD00000023054AD3
:103CC00019460133102BC2E9001102F10802F8D1A4
:103CD000704700BFD0380220034611F8012B03F8CB
:103CE000012B002AF9D1704753544D3332463F3FE0
:103CF0003F3F3F3F0053544D333246375B347C35B2
:103D00005D780053544D333246375B367C375D78EF
:103D100000000000D02C0220D423022040240220E6
:103D2000AC2402200096000000000000000000000B
:103D30000000000000000000000000000000000083
:103D40009515000881150008BD150008A915000883
:103D5000B5150008A11500088D1500087915000893
:103D6000C915000800000000A11600088D16000803
:103D7000C9160008B5160008C1160008AD160008DF
:103D80009916000885160008D516000800000000E6
:103D900001000000000000006D61696E000000007D
:103DA00069646C6500000000A03D0008582B0220EB
:103DB000D02C0220010000000120000800000000BB
:103DC0004865782F50726F6669434E430025424F15
:103DD000415244252D424C002553455249414C2522
:103DE000000000000200000000000000BD180008F4
:103DF000291900084000400078350220883502204B
:103E000002000000000000000300000000000000AD
:103E10006D19000800000000100000009835022015
:103E200000000000010000000000000040380220F7
:103E300001010200F1230008012300089D2300086E
:103E400081230008430000004C3E000809024300A3
:103E5000020100C032090400000102020100052431
:103E600000100105240100010424020205240600BB
:103E700001070582030800FF09040100020A00008F
:103E80000007050102400000070581024000000014
:103E900012000000983E00081201100102000040CC
:103EA000AE2D021000020102030100000403090408
:103EB00025424F41524425004375626559656C6C3B
:103EC0006F772D626473686F74003031323334352C
:103ED00036373839414243444546000000800000EF
:103EE0000080000000800000008000000000020050
:103EF00000000400000004000000040000000400B2
:103F000000000400000004000000040000000000A5
:103F1000B51A00086D1D0008191E00084000400079
:103F2000B8380220B838022001000000C83802204A
:103F30008000000040010000050000000000802A11
:103F400000000000AAAAAAAA00000024FFFF0000A7
:103F50000000000000A00A000001000000000000B6
:103F6000AAAAAAAA00000000FFFF000000000000AB
:103F7000000000001400005400000000AAAAAAAA31
:103F800014000054FFFF00000000000000000000CB
:103F900080699A0100000000AAAA8AAA405555012A
:103FA000FFFF0000007070077770000000810200C2
:103FB00000000000AAAAAAAA00410100FFFF000019
:103FC0000000008008000000000000000000000069
:103FD000AAAAAAAA00000000FFFF0000000000003B
:103FE000000000000000000000000000AAAAAAAA29
:103FF00000000000FFFF00000000000000000000C3
:104000000000000000000000AAAAAAAA0000000008
:10401000FFFF0000000000000000000000000000A2
:1040200000000000AAAAAAAA00000000FFFF0000EA
:104030000000000000000000000000000000000080
:10404000AAAAAAAA00000000FFFF000000000000CA
:10405000000000000000000000000000AAAA00000C
:1040600000000000FF000000000000000000000051
:10407000780000000000000000801E00000000002A
:10408000FF00000000000000E83C00083F000000C6
:1040900049040000F53C00083F0000005104000006
:1040A000033D00083F0000000096000000000800EB
:1040B000960000000008000004000000AC3E00086C
:1040C00000000000000000000000000000000000F0
:0840D0000000000000000000E8
:00000001FF
